:020000040030CA
:0E00000000C80F000080800003C003E0034032
:020000040000FA
:020000001FD00F
:020000040000FA
:10004000E0D09EBA01D0FDD7ABA203D0AB98AB886D
:10005000F8D7EC6EAE50ABA402D0ED50F2D7120040
:10006000ACB201D0FDD7AD6EED501200050022D824
:10007000FE6EED50FD6EED501200EC6E000EAFD036
:10008000A68EA69C7DD8F9D7A68EA69C7CD8F5D73F
:100090000F0B82D8F2D714D00FD014D04BD050D041
:1000A000ECD7FF0028D01CD03BD02FD04FD05AD057
:1000B000E7D7EAD780D87FD0EC6E010E90D88FD0EA
:1000C0007AD8DBD7D3DFD9D776D8FF0FED5002E34C
:1000D00072D8DEDF1200F8DFFED76DD8EC6E7FD06D
:1000E000FCDFE46EED50EC6E0900F55078D8E706C1
:1000F000FAE1E5521200F1DFE46EED50EC6EDE50F5
:100100006ED8E706FBE1E552120055D8E46EED50DB
:1001100052D8F56E0D00ED50E706FAE1E552ADD785
:100120004AD8E46EED5047D8DE6EED50E706FBE1AD
:10013000E552A3D7BFDFDA6EED50D96EED509DD7F3
:10014000B9DFF76EED50F66EED5097D7EC6E400EBE
:10015000E46EFF0EEC6E0900F550ED14E706FAE1CF
:10016000E552AAD7EC6EE950800FA6D7EC6EF29E4E
:10017000550EA76EAA0EA76EA682F28EED50120043
:10018000A684A688F3D7A684A6980A00EFDF090004
:100190001200EF60EF6EED50E844FD26010BFE22E9
:1001A000ED50120000D8EC6E450EE46EED50E706FF
:1001B000FEE1E552120081AC01D0FDD7F4DFF2DFA1
:1001C000EC6E080EE46E000E81AC02D0D88001D037
:1001D000D890E830E7DFE706F7E1E55212008A9EA3
:1001E000E1DFEC6E080EE46EED50E83002E38A8E3B
:1001F00001D08A9ED7DFE706F8E1E5528A8EED50FE
:10020000D1D7000EFC6E00EE7FF010EE8FF08A6802
:0E021000EC6E700ED36E938C939EED505CD707
:00000001FF
